Archive member included to satisfy reference by file (symbol)

d:/ahl-gec-ide(4.20)/gcc/bin/../lib/gcc/arm-none-eabi/7.2.1/../../../../arm-none-eabi/lib/thumb/v7e-m/fpv4-sp/hard\libc_nano.a(lib_a-exit.o)
                              d:/ahl-gec-ide(4.20)/gcc/bin/../lib/gcc/arm-none-eabi/7.2.1/../../../../arm-none-eabi/lib/thumb/v7e-m/fpv4-sp/hard/crt0.o (exit)
d:/ahl-gec-ide(4.20)/gcc/bin/../lib/gcc/arm-none-eabi/7.2.1/../../../../arm-none-eabi/lib/thumb/v7e-m/fpv4-sp/hard\libc_nano.a(lib_a-impure.o)
                              d:/ahl-gec-ide(4.20)/gcc/bin/../lib/gcc/arm-none-eabi/7.2.1/../../../../arm-none-eabi/lib/thumb/v7e-m/fpv4-sp/hard\libc_nano.a(lib_a-exit.o) (_global_impure_ptr)
d:/ahl-gec-ide(4.20)/gcc/bin/../lib/gcc/arm-none-eabi/7.2.1/../../../../arm-none-eabi/lib/thumb/v7e-m/fpv4-sp/hard\libc_nano.a(lib_a-init.o)
                              d:/ahl-gec-ide(4.20)/gcc/bin/../lib/gcc/arm-none-eabi/7.2.1/../../../../arm-none-eabi/lib/thumb/v7e-m/fpv4-sp/hard/crt0.o (__libc_init_array)
d:/ahl-gec-ide(4.20)/gcc/bin/../lib/gcc/arm-none-eabi/7.2.1/../../../../arm-none-eabi/lib/thumb/v7e-m/fpv4-sp/hard\libc_nano.a(lib_a-memcpy-stub.o)
                              ./obj/flash.o (memcpy)
d:/ahl-gec-ide(4.20)/gcc/bin/../lib/gcc/arm-none-eabi/7.2.1/../../../../arm-none-eabi/lib/thumb/v7e-m/fpv4-sp/hard\libc_nano.a(lib_a-memset.o)
                              d:/ahl-gec-ide(4.20)/gcc/bin/../lib/gcc/arm-none-eabi/7.2.1/../../../../arm-none-eabi/lib/thumb/v7e-m/fpv4-sp/hard/crt0.o (memset)
d:/ahl-gec-ide(4.20)/gcc/bin/../lib/gcc/arm-none-eabi/7.2.1/../../../../arm-none-eabi/lib/thumb/v7e-m/fpv4-sp/hard\libc_nano.a(lib_a-strcmp.o)
                              ./obj/emuart.o (strcmp)
d:/ahl-gec-ide(4.20)/gcc/bin/../lib/gcc/arm-none-eabi/7.2.1/../../../../arm-none-eabi/lib/thumb/v7e-m/fpv4-sp/hard\libc_nano.a(lib_a-strlen.o)
                              ./obj/printf.o (strlen)
d:/ahl-gec-ide(4.20)/gcc/bin/../lib/gcc/arm-none-eabi/7.2.1/../../../../arm-none-eabi/lib/thumb/v7e-m/fpv4-sp/hard\libc_nano.a(lib_a-strncmp.o)
                              ./obj/emuart.o (strncmp)
d:/ahl-gec-ide(4.20)/gcc/bin/../lib/gcc/arm-none-eabi/7.2.1/thumb/v7e-m/fpv4-sp/hard\libgcc.a(_arm_addsubdf3.o)
                              ./obj/uart.o (__aeabi_dsub)
d:/ahl-gec-ide(4.20)/gcc/bin/../lib/gcc/arm-none-eabi/7.2.1/thumb/v7e-m/fpv4-sp/hard\libgcc.a(_arm_muldivdf3.o)
                              ./obj/pwm.o (__aeabi_dmul)
d:/ahl-gec-ide(4.20)/gcc/bin/../lib/gcc/arm-none-eabi/7.2.1/thumb/v7e-m/fpv4-sp/hard\libgcc.a(_arm_cmpdf2.o)
                              ./obj/printf.o (__aeabi_dcmplt)
d:/ahl-gec-ide(4.20)/gcc/bin/../lib/gcc/arm-none-eabi/7.2.1/thumb/v7e-m/fpv4-sp/hard\libgcc.a(_arm_fixunsdfsi.o)
                              ./obj/pwm.o (__aeabi_d2uiz)
d:/ahl-gec-ide(4.20)/gcc/bin/../lib/gcc/arm-none-eabi/7.2.1/thumb/v7e-m/fpv4-sp/hard\libgcc.a(_aeabi_uldivmod.o)
                              ./obj/printf.o (__aeabi_uldivmod)
d:/ahl-gec-ide(4.20)/gcc/bin/../lib/gcc/arm-none-eabi/7.2.1/thumb/v7e-m/fpv4-sp/hard\libgcc.a(_fixunsdfdi.o)
                              ./obj/printf.o (__aeabi_d2ulz)
d:/ahl-gec-ide(4.20)/gcc/bin/../lib/gcc/arm-none-eabi/7.2.1/thumb/v7e-m/fpv4-sp/hard\libgcc.a(_udivmoddi4.o)
                              d:/ahl-gec-ide(4.20)/gcc/bin/../lib/gcc/arm-none-eabi/7.2.1/thumb/v7e-m/fpv4-sp/hard\libgcc.a(_aeabi_uldivmod.o) (__udivmoddi4)
d:/ahl-gec-ide(4.20)/gcc/bin/../lib/gcc/arm-none-eabi/7.2.1/thumb/v7e-m/fpv4-sp/hard\libgcc.a(_dvmd_tls.o)
                              d:/ahl-gec-ide(4.20)/gcc/bin/../lib/gcc/arm-none-eabi/7.2.1/thumb/v7e-m/fpv4-sp/hard\libgcc.a(_aeabi_uldivmod.o) (__aeabi_ldiv0)
d:/ahl-gec-ide(4.20)/gcc/bin/../lib/gcc/arm-none-eabi/7.2.1/../../../../arm-none-eabi/lib/thumb/v7e-m/fpv4-sp/hard\libnosys.a(_exit.o)
                              d:/ahl-gec-ide(4.20)/gcc/bin/../lib/gcc/arm-none-eabi/7.2.1/../../../../arm-none-eabi/lib/thumb/v7e-m/fpv4-sp/hard\libc_nano.a(lib_a-exit.o) (_exit)

Allocating common symbols
Common symbol       size              file

gTime               0x3               ./obj/main.o
component_fun       0x4               ./obj/startup_msp432p401r_gcc.o
gcRecvLen           0x2               ./obj/main.o
gcRecvDCLen         0x2               ./obj/main.o
gcRecvBuf           0x1000            ./obj/main.o

Discarded input sections

 .fini_array    0x00000000        0x4 d:/ahl-gec-ide(4.20)/gcc/bin/../lib/gcc/arm-none-eabi/7.2.1/thumb/v7e-m/fpv4-sp/hard/crtbegin.o
 .ARM.extab     0x00000000        0x0 d:/ahl-gec-ide(4.20)/gcc/bin/../lib/gcc/arm-none-eabi/7.2.1/../../../../arm-none-eabi/lib/thumb/v7e-m/fpv4-sp/hard/crt0.o
 .ARM.extab     0x00000000        0x0 d:/ahl-gec-ide(4.20)/gcc/bin/../lib/gcc/arm-none-eabi/7.2.1/thumb/v7e-m/fpv4-sp/hard\libgcc.a(_udivmoddi4.o)
 .eh_frame      0x00000000        0x4 d:/ahl-gec-ide(4.20)/gcc/bin/../lib/gcc/arm-none-eabi/7.2.1/thumb/v7e-m/fpv4-sp/hard/crtend.o
 .init          0x00000000        0x8 d:/ahl-gec-ide(4.20)/gcc/bin/../lib/gcc/arm-none-eabi/7.2.1/thumb/v7e-m/fpv4-sp/hard/crtn.o
 .fini          0x00000000        0x8 d:/ahl-gec-ide(4.20)/gcc/bin/../lib/gcc/arm-none-eabi/7.2.1/thumb/v7e-m/fpv4-sp/hard/crtn.o

Memory Configuration

Name             Origin             Length             Attributes
USER_INTVEC      0x0001a000         0x00001000         xr
MAIN_FLASH       0x0001b000         0x00025000         xr
SRAM_DATA        0x20002000         0x0000e000         rw
*default*        0x00000000         0xffffffff

Linker script and memory map

LOAD d:/ahl-gec-ide(4.20)/gcc/bin/../lib/gcc/arm-none-eabi/7.2.1/thumb/v7e-m/fpv4-sp/hard/crti.o
LOAD d:/ahl-gec-ide(4.20)/gcc/bin/../lib/gcc/arm-none-eabi/7.2.1/thumb/v7e-m/fpv4-sp/hard/crtbegin.o
LOAD d:/ahl-gec-ide(4.20)/gcc/bin/../lib/gcc/arm-none-eabi/7.2.1/../../../../arm-none-eabi/lib/thumb/v7e-m/fpv4-sp/hard/crt0.o
LOAD ./obj/emuart.o
LOAD ./obj/systick.o
LOAD ./obj/system_msp432p401r.o
LOAD ./obj/startup_msp432p401r_gcc.o
LOAD ./obj/main.o
LOAD ./obj/flash.o
LOAD ./obj/gpio.o
LOAD ./obj/wdog.o
LOAD ./obj/pwm.o
LOAD ./obj/gec.o
LOAD ./obj/uart.o
LOAD ./obj/isr.o
LOAD ./obj/printf.o
START GROUP
LOAD d:/ahl-gec-ide(4.20)/gcc/bin/../lib/gcc/arm-none-eabi/7.2.1/../../../../arm-none-eabi/lib/thumb/v7e-m/fpv4-sp/hard\libc_nano.a
LOAD d:/ahl-gec-ide(4.20)/gcc/bin/../lib/gcc/arm-none-eabi/7.2.1/../../../../arm-none-eabi/lib/thumb/v7e-m/fpv4-sp/hard\libm.a
END GROUP
START GROUP
LOAD d:/ahl-gec-ide(4.20)/gcc/bin/../lib/gcc/arm-none-eabi/7.2.1/thumb/v7e-m/fpv4-sp/hard\libgcc.a
LOAD d:/ahl-gec-ide(4.20)/gcc/bin/../lib/gcc/arm-none-eabi/7.2.1/../../../../arm-none-eabi/lib/thumb/v7e-m/fpv4-sp/hard\libc_nano.a
END GROUP
START GROUP
LOAD d:/ahl-gec-ide(4.20)/gcc/bin/../lib/gcc/arm-none-eabi/7.2.1/thumb/v7e-m/fpv4-sp/hard\libgcc.a
LOAD d:/ahl-gec-ide(4.20)/gcc/bin/../lib/gcc/arm-none-eabi/7.2.1/../../../../arm-none-eabi/lib/thumb/v7e-m/fpv4-sp/hard\libc_nano.a
LOAD d:/ahl-gec-ide(4.20)/gcc/bin/../lib/gcc/arm-none-eabi/7.2.1/../../../../arm-none-eabi/lib/thumb/v7e-m/fpv4-sp/hard\libnosys.a
END GROUP
START GROUP
LOAD d:/ahl-gec-ide(4.20)/gcc/bin/../lib/gcc/arm-none-eabi/7.2.1/thumb/v7e-m/fpv4-sp/hard\libgcc.a
LOAD d:/ahl-gec-ide(4.20)/gcc/bin/../lib/gcc/arm-none-eabi/7.2.1/../../../../arm-none-eabi/lib/thumb/v7e-m/fpv4-sp/hard\libc_nano.a
LOAD d:/ahl-gec-ide(4.20)/gcc/bin/../lib/gcc/arm-none-eabi/7.2.1/../../../../arm-none-eabi/lib/thumb/v7e-m/fpv4-sp/hard\libnosys.a
END GROUP
LOAD d:/ahl-gec-ide(4.20)/gcc/bin/../lib/gcc/arm-none-eabi/7.2.1/thumb/v7e-m/fpv4-sp/hard/crtend.o
LOAD d:/ahl-gec-ide(4.20)/gcc/bin/../lib/gcc/arm-none-eabi/7.2.1/thumb/v7e-m/fpv4-sp/hard/crtn.o
                0x00001000                MCU_SECTORSIZE = 0x1000
                0x00000000                MCU_FLASH_ADDR_START = 0x0
                0x0000001a                GEC_USER_SECTOR_START = 0x1a
                0x0000003f                GEC_USER_SECTOR_END = 0x3f
                0x20002000                GEC_USER_RAM_START = 0x20002000
                0x20010000                GEC_USER_RAM_END = 0x20010000
                0x0001a000                PROVIDE (_intvecs_base_address, DEFINED (_intvecs_base_address)?_intvecs_base_address:(MCU_SECTORSIZE * GEC_USER_SECTOR_START))

.intvecs        0x0001a000       0xe4
 *(.intvecs)
 .intvecs       0x0001a000       0xe4 ./obj/startup_msp432p401r_gcc.o
                0x0001a000                interruptVectors
                0x20002000                PROVIDE (_vtable_base_address, DEFINED (_vtable_base_address)?_vtable_base_address:GEC_USER_RAM_START)

.vtable
 *(.vtable)

.text           0x0001b000     0x50bc
 CREATE_OBJECT_SYMBOLS
 *(.text)
 .text          0x0001b000        0x0 d:/ahl-gec-ide(4.20)/gcc/bin/../lib/gcc/arm-none-eabi/7.2.1/thumb/v7e-m/fpv4-sp/hard/crti.o
 .text          0x0001b000       0x40 d:/ahl-gec-ide(4.20)/gcc/bin/../lib/gcc/arm-none-eabi/7.2.1/thumb/v7e-m/fpv4-sp/hard/crtbegin.o
 .text          0x0001b040       0x74 d:/ahl-gec-ide(4.20)/gcc/bin/../lib/gcc/arm-none-eabi/7.2.1/../../../../arm-none-eabi/lib/thumb/v7e-m/fpv4-sp/hard/crt0.o
                0x0001b040                _start
                0x0001b040                _mainCRTStartup
 .text          0x0001b0b4      0x6e8 ./obj/emuart.o
                0x0001b0b4                emuart_init
                0x0001b0e4                emuart_send1
                0x0001b100                emuart_sendN
                0x0001b11e                emuart_send_string
                0x0001b150                emuart_frame
                0x0001b3c4                useremuart_frame
                0x0001b660                sendFrame
                0x0001b724                crc16
 .text          0x0001b79c       0xa0 ./obj/systick.o
                0x0001b7f0                systick_init
 .text          0x0001b83c      0x3c8 ./obj/system_msp432p401r.o
                0x0001b83c                SystemCoreClockUpdate
                0x0001bb3c                SystemInit
 .text          0x0001bc04       0x6c ./obj/startup_msp432p401r_gcc.o
                0x0001bc04                Reset_Handler
                0x0001bc60                DebugMon_Handler
                0x0001bc60                AES256_IRQHandler
                0x0001bc60                HardFault_Handler
                0x0001bc60                PendSV_Handler
                0x0001bc60                NMI_Handler
                0x0001bc60                RTC_C_IRQHandler
                0x0001bc60                PORT1_IRQHandler
                0x0001bc60                FPU_IRQHandler
                0x0001bc60                PORT2_IRQHandler
                0x0001bc60                TA3_0_IRQHandler
                0x0001bc60                UsageFault_Handler
                0x0001bc60                DMA_INT3_IRQHandler
                0x0001bc60                TA2_0_IRQHandler
                0x0001bc60                DMA_INT1_IRQHandler
                0x0001bc60                WDT_A_IRQHandler
                0x0001bc60                TA2_N_IRQHandler
                0x0001bc60                TA1_0_IRQHandler
                0x0001bc60                CS_IRQHandler
                0x0001bc60                PSS_IRQHandler
                0x0001bc60                DMA_INT2_IRQHandler
                0x0001bc60                DMA_INT0_IRQHandler
                0x0001bc60                PORT4_IRQHandler
                0x0001bc60                PORT5_IRQHandler
                0x0001bc60                EUSCIB0_IRQHandler
                0x0001bc60                Default_Handler
                0x0001bc60                T32_INTC_IRQHandler
                0x0001bc60                TA3_N_IRQHandler
                0x0001bc60                TA0_0_IRQHandler
                0x0001bc60                EUSCIA2_IRQHandler
                0x0001bc60                PORT6_IRQHandler
                0x0001bc60                PORT3_IRQHandler
                0x0001bc60                MemManage_Handler
                0x0001bc60                SVC_Handler
                0x0001bc60                TA1_N_IRQHandler
                0x0001bc60                EUSCIA1_IRQHandler
                0x0001bc60                COMP_E1_IRQHandler
                0x0001bc60                EUSCIB2_IRQHandler
                0x0001bc60                FLCTL_IRQHandler
                0x0001bc60                EUSCIB3_IRQHandler
                0x0001bc60                T32_INT1_IRQHandler
                0x0001bc60                DMA_ERR_IRQHandler
                0x0001bc60                ADC14_IRQHandler
                0x0001bc60                EUSCIA0_IRQHandler
                0x0001bc60                BusFault_Handler
                0x0001bc60                PCM_IRQHandler
                0x0001bc60                TA0_N_IRQHandler
                0x0001bc60                COMP_E0_IRQHandler
                0x0001bc60                EUSCIB1_IRQHandler
                0x0001bc60                T32_INT2_IRQHandler
 .text          0x0001bc70      0x164 ./obj/main.o
                0x0001bc70                main
 .text          0x0001bdd4      0x830 ./obj/flash.o
                0x0001bdd4                flash_init
                0x0001be00                flash_erase
                0x0001bf54                flash_write
                0x0001c100                flash_write_physical
                0x0001c284                flash_read_physical
                0x0001c2aa                flash_read_logic
                0x0001c352                flash_protect
                0x0001c40c                flash_unprotect
                0x0001c4cc                flash_isSectorProtected
                0x0001c54c                flash_isempty
 .text          0x0001c604      0xc58 ./obj/gpio.o
                0x0001c69a                gpio_init
                0x0001c96c                gpio_set
                0x0001caac                gpio_get
                0x0001cb6c                gpio_reverse
                0x0001ccd4                gpio_pull
                0x0001ce14                gpio_enable_int
                0x0001cfcc                gpio_disable_int
                0x0001d0bc                gpio_drive_strength
 .text          0x0001d25c       0xf8 ./obj/wdog.o
                0x0001d25c                wdog_start
                0x0001d31c                wdog_stop
                0x0001d338                wdog_feed
 .text          0x0001d354      0x62c ./obj/pwm.o
                0x0001d354                pwm_init
                0x0001d7bc                pwm_update
                0x0001d8ac                tpm_mux_val
 .text          0x0001d980      0x394 ./obj/gec.o
                0x0001d9a8                Vectors_Init
                0x0001da7c                SYSTEM_FUNCTION
 *fill*         0x0001dd14        0x4 
 .text          0x0001dd18      0x640 ./obj/uart.o
                0x0001dd80                uart_init
                0x0001dfa0                uart_send1
                0x0001e018                uart_sendN
                0x0001e080                uart_send_string
                0x0001e0e4                uart_re1
                0x0001e168                uart_reN
                0x0001e1d6                uart_enable_re_int
                0x0001e228                uart_disable_re_int
                0x0001e278                uart_get_re_int
                0x0001e2c8                uart_is_uartNo
                0x0001e2ea                BRSxSel
 .text          0x0001e358      0x180 ./obj/isr.o
                0x0001e358                EUSCIA3_IRQHandler
                0x0001e3a6                SysTick_Handler
                0x0001e3dc                User_SysFun
                0x0001e458                SecAdd1
 .text          0x0001e4d8      0xec4 ./obj/printf.o
                0x0001e4d8                out_char
                0x0001e544                printk_mkfloatstr
                0x0001e9c2                printk
                0x0001f360                myprintf
 .text          0x0001f39c        0x0 d:/ahl-gec-ide(4.20)/gcc/bin/../lib/gcc/arm-none-eabi/7.2.1/../../../../arm-none-eabi/lib/thumb/v7e-m/fpv4-sp/hard\libc_nano.a(lib_a-exit.o)
 .text          0x0001f39c        0x0 d:/ahl-gec-ide(4.20)/gcc/bin/../lib/gcc/arm-none-eabi/7.2.1/../../../../arm-none-eabi/lib/thumb/v7e-m/fpv4-sp/hard\libc_nano.a(lib_a-impure.o)
 .text          0x0001f39c        0x0 d:/ahl-gec-ide(4.20)/gcc/bin/../lib/gcc/arm-none-eabi/7.2.1/../../../../arm-none-eabi/lib/thumb/v7e-m/fpv4-sp/hard\libc_nano.a(lib_a-init.o)
 .text          0x0001f39c        0x0 d:/ahl-gec-ide(4.20)/gcc/bin/../lib/gcc/arm-none-eabi/7.2.1/../../../../arm-none-eabi/lib/thumb/v7e-m/fpv4-sp/hard\libc_nano.a(lib_a-memcpy-stub.o)
 .text          0x0001f39c        0x0 d:/ahl-gec-ide(4.20)/gcc/bin/../lib/gcc/arm-none-eabi/7.2.1/../../../../arm-none-eabi/lib/thumb/v7e-m/fpv4-sp/hard\libc_nano.a(lib_a-memset.o)
 .text          0x0001f39c       0x14 d:/ahl-gec-ide(4.20)/gcc/bin/../lib/gcc/arm-none-eabi/7.2.1/../../../../arm-none-eabi/lib/thumb/v7e-m/fpv4-sp/hard\libc_nano.a(lib_a-strcmp.o)
                0x0001f39c                strcmp
 .text          0x0001f3b0       0x10 d:/ahl-gec-ide(4.20)/gcc/bin/../lib/gcc/arm-none-eabi/7.2.1/../../../../arm-none-eabi/lib/thumb/v7e-m/fpv4-sp/hard\libc_nano.a(lib_a-strlen.o)
                0x0001f3b0                strlen
 .text          0x0001f3c0        0x0 d:/ahl-gec-ide(4.20)/gcc/bin/../lib/gcc/arm-none-eabi/7.2.1/../../../../arm-none-eabi/lib/thumb/v7e-m/fpv4-sp/hard\libc_nano.a(lib_a-strncmp.o)
 .text          0x0001f3c0      0x378 d:/ahl-gec-ide(4.20)/gcc/bin/../lib/gcc/arm-none-eabi/7.2.1/thumb/v7e-m/fpv4-sp/hard\libgcc.a(_arm_addsubdf3.o)
                0x0001f3c0                __aeabi_drsub
                0x0001f3c8                __aeabi_dsub
                0x0001f3c8                __subdf3
                0x0001f3cc                __aeabi_dadd
                0x0001f3cc                __adddf3
                0x0001f644                __floatunsidf
                0x0001f644                __aeabi_ui2d
                0x0001f664                __floatsidf
                0x0001f664                __aeabi_i2d
                0x0001f688                __aeabi_f2d
                0x0001f688                __extendsfdf2
                0x0001f6cc                __floatundidf
                0x0001f6cc                __aeabi_ul2d
                0x0001f6dc                __floatdidf
                0x0001f6dc                __aeabi_l2d
 .text          0x0001f738      0x424 d:/ahl-gec-ide(4.20)/gcc/bin/../lib/gcc/arm-none-eabi/7.2.1/thumb/v7e-m/fpv4-sp/hard\libgcc.a(_arm_muldivdf3.o)
                0x0001f738                __aeabi_dmul
                0x0001f738                __muldf3
                0x0001f98c                __divdf3
                0x0001f98c                __aeabi_ddiv
 .text          0x0001fb5c      0x110 d:/ahl-gec-ide(4.20)/gcc/bin/../lib/gcc/arm-none-eabi/7.2.1/thumb/v7e-m/fpv4-sp/hard\libgcc.a(_arm_cmpdf2.o)
                0x0001fb5c                __gtdf2
                0x0001fb5c                __gedf2
                0x0001fb64                __ltdf2
                0x0001fb64                __ledf2
                0x0001fb6c                __nedf2
                0x0001fb6c                __eqdf2
                0x0001fb6c                __cmpdf2
                0x0001fbe8                __aeabi_cdrcmple
                0x0001fbf8                __aeabi_cdcmpeq
                0x0001fbf8                __aeabi_cdcmple
                0x0001fc08                __aeabi_dcmpeq
                0x0001fc1c                __aeabi_dcmplt
                0x0001fc30                __aeabi_dcmple
                0x0001fc44                __aeabi_dcmpge
                0x0001fc58                __aeabi_dcmpgt
 .text          0x0001fc6c       0x40 d:/ahl-gec-ide(4.20)/gcc/bin/../lib/gcc/arm-none-eabi/7.2.1/thumb/v7e-m/fpv4-sp/hard\libgcc.a(_arm_fixunsdfsi.o)
                0x0001fc6c                __aeabi_d2uiz
                0x0001fc6c                __fixunsdfsi
 .text          0x0001fcac       0x30 d:/ahl-gec-ide(4.20)/gcc/bin/../lib/gcc/arm-none-eabi/7.2.1/thumb/v7e-m/fpv4-sp/hard\libgcc.a(_aeabi_uldivmod.o)
                0x0001fcac                __aeabi_uldivmod
 .text          0x0001fcdc       0x44 d:/ahl-gec-ide(4.20)/gcc/bin/../lib/gcc/arm-none-eabi/7.2.1/thumb/v7e-m/fpv4-sp/hard\libgcc.a(_fixunsdfdi.o)
                0x0001fcdc                __fixunsdfdi
                0x0001fcdc                __aeabi_d2ulz
 .text          0x0001fd20      0x2cc d:/ahl-gec-ide(4.20)/gcc/bin/../lib/gcc/arm-none-eabi/7.2.1/thumb/v7e-m/fpv4-sp/hard\libgcc.a(_udivmoddi4.o)
                0x0001fd20                __udivmoddi4
 .text          0x0001ffec        0x4 d:/ahl-gec-ide(4.20)/gcc/bin/../lib/gcc/arm-none-eabi/7.2.1/thumb/v7e-m/fpv4-sp/hard\libgcc.a(_dvmd_tls.o)
                0x0001ffec                __aeabi_idiv0
                0x0001ffec                __aeabi_ldiv0
 .text          0x0001fff0        0x0 d:/ahl-gec-ide(4.20)/gcc/bin/../lib/gcc/arm-none-eabi/7.2.1/../../../../arm-none-eabi/lib/thumb/v7e-m/fpv4-sp/hard\libnosys.a(_exit.o)
 .text          0x0001fff0        0x0 d:/ahl-gec-ide(4.20)/gcc/bin/../lib/gcc/arm-none-eabi/7.2.1/thumb/v7e-m/fpv4-sp/hard/crtend.o
 .text          0x0001fff0        0x0 d:/ahl-gec-ide(4.20)/gcc/bin/../lib/gcc/arm-none-eabi/7.2.1/thumb/v7e-m/fpv4-sp/hard/crtn.o
 *(.text.*)
 .text.exit     0x0001fff0       0x28 d:/ahl-gec-ide(4.20)/gcc/bin/../lib/gcc/arm-none-eabi/7.2.1/../../../../arm-none-eabi/lib/thumb/v7e-m/fpv4-sp/hard\libc_nano.a(lib_a-exit.o)
                0x0001fff0                exit
 .text.__libc_init_array
                0x00020018       0x48 d:/ahl-gec-ide(4.20)/gcc/bin/../lib/gcc/arm-none-eabi/7.2.1/../../../../arm-none-eabi/lib/thumb/v7e-m/fpv4-sp/hard\libc_nano.a(lib_a-init.o)
                0x00020018                __libc_init_array
 .text.memcpy   0x00020060       0x16 d:/ahl-gec-ide(4.20)/gcc/bin/../lib/gcc/arm-none-eabi/7.2.1/../../../../arm-none-eabi/lib/thumb/v7e-m/fpv4-sp/hard\libc_nano.a(lib_a-memcpy-stub.o)
                0x00020060                memcpy
 .text.memset   0x00020076       0x10 d:/ahl-gec-ide(4.20)/gcc/bin/../lib/gcc/arm-none-eabi/7.2.1/../../../../arm-none-eabi/lib/thumb/v7e-m/fpv4-sp/hard\libc_nano.a(lib_a-memset.o)
                0x00020076                memset
 .text.strncmp  0x00020086       0x24 d:/ahl-gec-ide(4.20)/gcc/bin/../lib/gcc/arm-none-eabi/7.2.1/../../../../arm-none-eabi/lib/thumb/v7e-m/fpv4-sp/hard\libc_nano.a(lib_a-strncmp.o)
                0x00020086                strncmp
 *fill*         0x000200aa        0x2 
 .text._exit    0x000200ac        0x4 d:/ahl-gec-ide(4.20)/gcc/bin/../lib/gcc/arm-none-eabi/7.2.1/../../../../arm-none-eabi/lib/thumb/v7e-m/fpv4-sp/hard\libnosys.a(_exit.o)
                0x000200ac                _exit
                0x000200b0                . = ALIGN (0x4)
 *(.ctors)
                0x000200b0                . = ALIGN (0x4)
 *(.dtors)
                0x000200b0                . = ALIGN (0x4)
                0x000200b0                __init_array_start = .
 *(.init_array*)
 .init_array    0x000200b0        0x4 d:/ahl-gec-ide(4.20)/gcc/bin/../lib/gcc/arm-none-eabi/7.2.1/thumb/v7e-m/fpv4-sp/hard/crtbegin.o
                0x000200b4                __init_array_end = .
 *(.init)
 .init          0x000200b4        0x4 d:/ahl-gec-ide(4.20)/gcc/bin/../lib/gcc/arm-none-eabi/7.2.1/thumb/v7e-m/fpv4-sp/hard/crti.o
                0x000200b4                _init
 *(.fini*)
 .fini          0x000200b8        0x4 d:/ahl-gec-ide(4.20)/gcc/bin/../lib/gcc/arm-none-eabi/7.2.1/thumb/v7e-m/fpv4-sp/hard/crti.o
                0x000200b8                _fini

.glue_7         0x000200bc        0x0
 .glue_7        0x000200bc        0x0 linker stubs

.glue_7t        0x000200bc        0x0
 .glue_7t       0x000200bc        0x0 linker stubs

.vfp11_veneer   0x000200bc        0x0
 .vfp11_veneer  0x000200bc        0x0 linker stubs

.v4_bx          0x000200bc        0x0
 .v4_bx         0x000200bc        0x0 linker stubs

.iplt           0x000200bc        0x0
 .iplt          0x000200bc        0x0 d:/ahl-gec-ide(4.20)/gcc/bin/../lib/gcc/arm-none-eabi/7.2.1/thumb/v7e-m/fpv4-sp/hard/crtbegin.o

.rodata         0x000200bc      0x1d0
 *(.rodata)
 .rodata        0x000200bc       0x2f ./obj/emuart.o
 *fill*         0x000200eb        0x1 
 .rodata        0x000200ec      0x116 ./obj/main.o
 *fill*         0x00020202        0x2 
 .rodata        0x00020204       0x7f ./obj/gec.o
 *fill*         0x00020283        0x1 
 .rodata        0x00020284        0x4 ./obj/uart.o
 *(.rodata.*)
 .rodata._global_impure_ptr
                0x00020288        0x4 d:/ahl-gec-ide(4.20)/gcc/bin/../lib/gcc/arm-none-eabi/7.2.1/../../../../arm-none-eabi/lib/thumb/v7e-m/fpv4-sp/hard\libc_nano.a(lib_a-impure.o)
                0x00020288                _global_impure_ptr

.eh_frame       0x0002028c        0x0
 .eh_frame      0x0002028c        0x0 d:/ahl-gec-ide(4.20)/gcc/bin/../lib/gcc/arm-none-eabi/7.2.1/thumb/v7e-m/fpv4-sp/hard/crtbegin.o

.ARM.exidx      0x0002028c        0x8
                0x0002028c                __exidx_start = .
 *(.ARM.exidx* .gnu.linkonce.armexidx.*)
 .ARM.exidx     0x0002028c        0x8 d:/ahl-gec-ide(4.20)/gcc/bin/../lib/gcc/arm-none-eabi/7.2.1/../../../../arm-none-eabi/lib/thumb/v7e-m/fpv4-sp/hard/crt0.o
 .ARM.exidx     0x00020294        0x0 d:/ahl-gec-ide(4.20)/gcc/bin/../lib/gcc/arm-none-eabi/7.2.1/thumb/v7e-m/fpv4-sp/hard\libgcc.a(_udivmoddi4.o)
                                  0x8 (size before relaxing)
                0x00020294                __exidx_end = .

.rel.dyn        0x00020294        0x0
 .rel.iplt      0x00020294        0x0 d:/ahl-gec-ide(4.20)/gcc/bin/../lib/gcc/arm-none-eabi/7.2.1/thumb/v7e-m/fpv4-sp/hard/crtbegin.o

.ARM.extab
 *(.ARM.extab* .gnu.linkonce.armextab.*)
                0x00020294                __etext = .

.data           0x20002000      0x16c load address 0x00020294
                0x00020294                __data_load__ = LOADADDR (.data)
                0x20002000                __data_start__ = .
 *(.data)
 .data          0x20002000        0x0 d:/ahl-gec-ide(4.20)/gcc/bin/../lib/gcc/arm-none-eabi/7.2.1/thumb/v7e-m/fpv4-sp/hard/crti.o
 .data          0x20002000        0x4 d:/ahl-gec-ide(4.20)/gcc/bin/../lib/gcc/arm-none-eabi/7.2.1/thumb/v7e-m/fpv4-sp/hard/crtbegin.o
                0x20002000                __dso_handle
 .data          0x20002004        0x0 d:/ahl-gec-ide(4.20)/gcc/bin/../lib/gcc/arm-none-eabi/7.2.1/../../../../arm-none-eabi/lib/thumb/v7e-m/fpv4-sp/hard/crt0.o
 .data          0x20002004       0x24 ./obj/emuart.o
 .data          0x20002028        0x0 ./obj/systick.o
 .data          0x20002028        0x4 ./obj/system_msp432p401r.o
                0x20002028                SystemCoreClock
 .data          0x2000202c        0x0 ./obj/startup_msp432p401r_gcc.o
 .data          0x2000202c        0x0 ./obj/main.o
 .data          0x2000202c        0x0 ./obj/flash.o
 .data          0x2000202c       0x28 ./obj/gpio.o
                0x2000202c                GPIO_ODD_ARR
                0x20002040                GPIO_EVEN_ARR
 .data          0x20002054        0x0 ./obj/wdog.o
 .data          0x20002054       0x38 ./obj/pwm.o
 .data          0x2000208c        0x0 ./obj/gec.o
 .data          0x2000208c       0x7c ./obj/uart.o
                0x2000209c                BRSxS
                0x200020e4                ValBRSxS
 .data          0x20002108        0x0 ./obj/isr.o
 .data          0x20002108        0x0 ./obj/printf.o
 .data          0x20002108        0x0 d:/ahl-gec-ide(4.20)/gcc/bin/../lib/gcc/arm-none-eabi/7.2.1/../../../../arm-none-eabi/lib/thumb/v7e-m/fpv4-sp/hard\libc_nano.a(lib_a-exit.o)
 .data          0x20002108        0x0 d:/ahl-gec-ide(4.20)/gcc/bin/../lib/gcc/arm-none-eabi/7.2.1/../../../../arm-none-eabi/lib/thumb/v7e-m/fpv4-sp/hard\libc_nano.a(lib_a-impure.o)
 .data          0x20002108        0x0 d:/ahl-gec-ide(4.20)/gcc/bin/../lib/gcc/arm-none-eabi/7.2.1/../../../../arm-none-eabi/lib/thumb/v7e-m/fpv4-sp/hard\libc_nano.a(lib_a-init.o)
 .data          0x20002108        0x0 d:/ahl-gec-ide(4.20)/gcc/bin/../lib/gcc/arm-none-eabi/7.2.1/../../../../arm-none-eabi/lib/thumb/v7e-m/fpv4-sp/hard\libc_nano.a(lib_a-memcpy-stub.o)
 .data          0x20002108        0x0 d:/ahl-gec-ide(4.20)/gcc/bin/../lib/gcc/arm-none-eabi/7.2.1/../../../../arm-none-eabi/lib/thumb/v7e-m/fpv4-sp/hard\libc_nano.a(lib_a-memset.o)
 .data          0x20002108        0x0 d:/ahl-gec-ide(4.20)/gcc/bin/../lib/gcc/arm-none-eabi/7.2.1/../../../../arm-none-eabi/lib/thumb/v7e-m/fpv4-sp/hard\libc_nano.a(lib_a-strcmp.o)
 .data          0x20002108        0x0 d:/ahl-gec-ide(4.20)/gcc/bin/../lib/gcc/arm-none-eabi/7.2.1/../../../../arm-none-eabi/lib/thumb/v7e-m/fpv4-sp/hard\libc_nano.a(lib_a-strlen.o)
 .data          0x20002108        0x0 d:/ahl-gec-ide(4.20)/gcc/bin/../lib/gcc/arm-none-eabi/7.2.1/../../../../arm-none-eabi/lib/thumb/v7e-m/fpv4-sp/hard\libc_nano.a(lib_a-strncmp.o)
 .data          0x20002108        0x0 d:/ahl-gec-ide(4.20)/gcc/bin/../lib/gcc/arm-none-eabi/7.2.1/thumb/v7e-m/fpv4-sp/hard\libgcc.a(_arm_addsubdf3.o)
 .data          0x20002108        0x0 d:/ahl-gec-ide(4.20)/gcc/bin/../lib/gcc/arm-none-eabi/7.2.1/thumb/v7e-m/fpv4-sp/hard\libgcc.a(_arm_muldivdf3.o)
 .data          0x20002108        0x0 d:/ahl-gec-ide(4.20)/gcc/bin/../lib/gcc/arm-none-eabi/7.2.1/thumb/v7e-m/fpv4-sp/hard\libgcc.a(_arm_cmpdf2.o)
 .data          0x20002108        0x0 d:/ahl-gec-ide(4.20)/gcc/bin/../lib/gcc/arm-none-eabi/7.2.1/thumb/v7e-m/fpv4-sp/hard\libgcc.a(_arm_fixunsdfsi.o)
 .data          0x20002108        0x0 d:/ahl-gec-ide(4.20)/gcc/bin/../lib/gcc/arm-none-eabi/7.2.1/thumb/v7e-m/fpv4-sp/hard\libgcc.a(_aeabi_uldivmod.o)
 .data          0x20002108        0x0 d:/ahl-gec-ide(4.20)/gcc/bin/../lib/gcc/arm-none-eabi/7.2.1/thumb/v7e-m/fpv4-sp/hard\libgcc.a(_fixunsdfdi.o)
 .data          0x20002108        0x0 d:/ahl-gec-ide(4.20)/gcc/bin/../lib/gcc/arm-none-eabi/7.2.1/thumb/v7e-m/fpv4-sp/hard\libgcc.a(_udivmoddi4.o)
 .data          0x20002108        0x0 d:/ahl-gec-ide(4.20)/gcc/bin/../lib/gcc/arm-none-eabi/7.2.1/thumb/v7e-m/fpv4-sp/hard\libgcc.a(_dvmd_tls.o)
 .data          0x20002108        0x0 d:/ahl-gec-ide(4.20)/gcc/bin/../lib/gcc/arm-none-eabi/7.2.1/../../../../arm-none-eabi/lib/thumb/v7e-m/fpv4-sp/hard\libnosys.a(_exit.o)
 .data          0x20002108        0x0 d:/ahl-gec-ide(4.20)/gcc/bin/../lib/gcc/arm-none-eabi/7.2.1/thumb/v7e-m/fpv4-sp/hard/crtend.o
 .data          0x20002108        0x0 d:/ahl-gec-ide(4.20)/gcc/bin/../lib/gcc/arm-none-eabi/7.2.1/thumb/v7e-m/fpv4-sp/hard/crtn.o
 *(.data*)
 .data._impure_ptr
                0x20002108        0x4 d:/ahl-gec-ide(4.20)/gcc/bin/../lib/gcc/arm-none-eabi/7.2.1/../../../../arm-none-eabi/lib/thumb/v7e-m/fpv4-sp/hard\libc_nano.a(lib_a-impure.o)
                0x20002108                _impure_ptr
 .data.impure_data
                0x2000210c       0x60 d:/ahl-gec-ide(4.20)/gcc/bin/../lib/gcc/arm-none-eabi/7.2.1/../../../../arm-none-eabi/lib/thumb/v7e-m/fpv4-sp/hard\libc_nano.a(lib_a-impure.o)
                0x2000216c                . = ALIGN (0x4)
                0x2000216c                __data_end__ = .

.igot.plt       0x2000216c        0x0 load address 0x00020400
 .igot.plt      0x2000216c        0x0 d:/ahl-gec-ide(4.20)/gcc/bin/../lib/gcc/arm-none-eabi/7.2.1/thumb/v7e-m/fpv4-sp/hard/crtbegin.o

.bss            0x2000216c     0x102c
                0x2000216c                __bss_start__ = .
 *(.shbss)
 *(.bss)
 .bss           0x2000216c        0x0 d:/ahl-gec-ide(4.20)/gcc/bin/../lib/gcc/arm-none-eabi/7.2.1/thumb/v7e-m/fpv4-sp/hard/crti.o
 .bss           0x2000216c       0x1c d:/ahl-gec-ide(4.20)/gcc/bin/../lib/gcc/arm-none-eabi/7.2.1/thumb/v7e-m/fpv4-sp/hard/crtbegin.o
 .bss           0x20002188        0x0 d:/ahl-gec-ide(4.20)/gcc/bin/../lib/gcc/arm-none-eabi/7.2.1/../../../../arm-none-eabi/lib/thumb/v7e-m/fpv4-sp/hard/crt0.o
 .bss           0x20002188        0x1 ./obj/emuart.o
 .bss           0x20002189        0x0 ./obj/systick.o
 .bss           0x20002189        0x0 ./obj/system_msp432p401r.o
 .bss           0x20002189        0x0 ./obj/startup_msp432p401r_gcc.o
 .bss           0x20002189        0x0 ./obj/main.o
 .bss           0x20002189        0x0 ./obj/flash.o
 .bss           0x20002189        0x0 ./obj/gpio.o
 .bss           0x20002189        0x0 ./obj/wdog.o
 .bss           0x20002189        0x0 ./obj/pwm.o
 .bss           0x20002189        0x0 ./obj/gec.o
 .bss           0x20002189        0x0 ./obj/uart.o
 .bss           0x20002189        0x1 ./obj/isr.o
 .bss           0x2000218a        0x0 ./obj/printf.o
 .bss           0x2000218a        0x0 d:/ahl-gec-ide(4.20)/gcc/bin/../lib/gcc/arm-none-eabi/7.2.1/../../../../arm-none-eabi/lib/thumb/v7e-m/fpv4-sp/hard\libc_nano.a(lib_a-exit.o)
 .bss           0x2000218a        0x0 d:/ahl-gec-ide(4.20)/gcc/bin/../lib/gcc/arm-none-eabi/7.2.1/../../../../arm-none-eabi/lib/thumb/v7e-m/fpv4-sp/hard\libc_nano.a(lib_a-impure.o)
 .bss           0x2000218a        0x0 d:/ahl-gec-ide(4.20)/gcc/bin/../lib/gcc/arm-none-eabi/7.2.1/../../../../arm-none-eabi/lib/thumb/v7e-m/fpv4-sp/hard\libc_nano.a(lib_a-init.o)
 .bss           0x2000218a        0x0 d:/ahl-gec-ide(4.20)/gcc/bin/../lib/gcc/arm-none-eabi/7.2.1/../../../../arm-none-eabi/lib/thumb/v7e-m/fpv4-sp/hard\libc_nano.a(lib_a-memcpy-stub.o)
 .bss           0x2000218a        0x0 d:/ahl-gec-ide(4.20)/gcc/bin/../lib/gcc/arm-none-eabi/7.2.1/../../../../arm-none-eabi/lib/thumb/v7e-m/fpv4-sp/hard\libc_nano.a(lib_a-memset.o)
 .bss           0x2000218a        0x0 d:/ahl-gec-ide(4.20)/gcc/bin/../lib/gcc/arm-none-eabi/7.2.1/../../../../arm-none-eabi/lib/thumb/v7e-m/fpv4-sp/hard\libc_nano.a(lib_a-strcmp.o)
 .bss           0x2000218a        0x0 d:/ahl-gec-ide(4.20)/gcc/bin/../lib/gcc/arm-none-eabi/7.2.1/../../../../arm-none-eabi/lib/thumb/v7e-m/fpv4-sp/hard\libc_nano.a(lib_a-strlen.o)
 .bss           0x2000218a        0x0 d:/ahl-gec-ide(4.20)/gcc/bin/../lib/gcc/arm-none-eabi/7.2.1/../../../../arm-none-eabi/lib/thumb/v7e-m/fpv4-sp/hard\libc_nano.a(lib_a-strncmp.o)
 .bss           0x2000218a        0x0 d:/ahl-gec-ide(4.20)/gcc/bin/../lib/gcc/arm-none-eabi/7.2.1/thumb/v7e-m/fpv4-sp/hard\libgcc.a(_arm_addsubdf3.o)
 .bss           0x2000218a        0x0 d:/ahl-gec-ide(4.20)/gcc/bin/../lib/gcc/arm-none-eabi/7.2.1/thumb/v7e-m/fpv4-sp/hard\libgcc.a(_arm_muldivdf3.o)
 .bss           0x2000218a        0x0 d:/ahl-gec-ide(4.20)/gcc/bin/../lib/gcc/arm-none-eabi/7.2.1/thumb/v7e-m/fpv4-sp/hard\libgcc.a(_arm_cmpdf2.o)
 .bss           0x2000218a        0x0 d:/ahl-gec-ide(4.20)/gcc/bin/../lib/gcc/arm-none-eabi/7.2.1/thumb/v7e-m/fpv4-sp/hard\libgcc.a(_arm_fixunsdfsi.o)
 .bss           0x2000218a        0x0 d:/ahl-gec-ide(4.20)/gcc/bin/../lib/gcc/arm-none-eabi/7.2.1/thumb/v7e-m/fpv4-sp/hard\libgcc.a(_aeabi_uldivmod.o)
 .bss           0x2000218a        0x0 d:/ahl-gec-ide(4.20)/gcc/bin/../lib/gcc/arm-none-eabi/7.2.1/thumb/v7e-m/fpv4-sp/hard\libgcc.a(_fixunsdfdi.o)
 .bss           0x2000218a        0x0 d:/ahl-gec-ide(4.20)/gcc/bin/../lib/gcc/arm-none-eabi/7.2.1/thumb/v7e-m/fpv4-sp/hard\libgcc.a(_udivmoddi4.o)
 .bss           0x2000218a        0x0 d:/ahl-gec-ide(4.20)/gcc/bin/../lib/gcc/arm-none-eabi/7.2.1/thumb/v7e-m/fpv4-sp/hard\libgcc.a(_dvmd_tls.o)
 .bss           0x2000218a        0x0 d:/ahl-gec-ide(4.20)/gcc/bin/../lib/gcc/arm-none-eabi/7.2.1/../../../../arm-none-eabi/lib/thumb/v7e-m/fpv4-sp/hard\libnosys.a(_exit.o)
 .bss           0x2000218a        0x0 d:/ahl-gec-ide(4.20)/gcc/bin/../lib/gcc/arm-none-eabi/7.2.1/thumb/v7e-m/fpv4-sp/hard/crtend.o
 .bss           0x2000218a        0x0 d:/ahl-gec-ide(4.20)/gcc/bin/../lib/gcc/arm-none-eabi/7.2.1/thumb/v7e-m/fpv4-sp/hard/crtn.o
 *(.bss.*)
 *(COMMON)
 *fill*         0x2000218a        0x2 
 COMMON         0x2000218c        0x4 ./obj/startup_msp432p401r_gcc.o
                0x2000218c                component_fun
 COMMON         0x20002190     0x1008 ./obj/main.o
                0x20002190                gTime
                0x20002194                gcRecvLen
                0x20002196                gcRecvDCLen
                0x20002198                gcRecvBuf
                0x20003198                . = ALIGN (0x4)
                0x20003198                __bss_end__ = .

.heap           0x20003198        0x0
                0x20003198                . = ALIGN (0x8)
                0x20003198                __end__ = .
                [!provide]                PROVIDE (end, .)
                0x20003198                __HeapBase = .
                0x20003198                __HeapLimit = .

.stack          0x20003198        0x0
                0x20003198                . = ALIGN (0x8)
                0x20010000                __StackTop = (ORIGIN (SRAM_DATA) + LENGTH (SRAM_DATA))
OUTPUT(PWMMSP432-20210406.out elf32-littlearm)

.ARM.attributes
                0x00000000       0x30
 .ARM.attributes
                0x00000000       0x22 d:/ahl-gec-ide(4.20)/gcc/bin/../lib/gcc/arm-none-eabi/7.2.1/thumb/v7e-m/fpv4-sp/hard/crti.o
 .ARM.attributes
                0x00000022       0x34 d:/ahl-gec-ide(4.20)/gcc/bin/../lib/gcc/arm-none-eabi/7.2.1/thumb/v7e-m/fpv4-sp/hard/crtbegin.o
 .ARM.attributes
                0x00000056       0x20 d:/ahl-gec-ide(4.20)/gcc/bin/../lib/gcc/arm-none-eabi/7.2.1/../../../../arm-none-eabi/lib/thumb/v7e-m/fpv4-sp/hard/crt0.o
 .ARM.attributes
                0x00000076       0x39 ./obj/emuart.o
 .ARM.attributes
                0x000000af       0x39 ./obj/systick.o
 .ARM.attributes
                0x000000e8       0x39 ./obj/system_msp432p401r.o
 .ARM.attributes
                0x00000121       0x39 ./obj/startup_msp432p401r_gcc.o
 .ARM.attributes
                0x0000015a       0x39 ./obj/main.o
 .ARM.attributes
                0x00000193       0x39 ./obj/flash.o
 .ARM.attributes
                0x000001cc       0x39 ./obj/gpio.o
 .ARM.attributes
                0x00000205       0x39 ./obj/wdog.o
 .ARM.attributes
                0x0000023e       0x39 ./obj/pwm.o
 .ARM.attributes
                0x00000277       0x39 ./obj/gec.o
 .ARM.attributes
                0x000002b0       0x39 ./obj/uart.o
 .ARM.attributes
                0x000002e9       0x39 ./obj/isr.o
 .ARM.attributes
                0x00000322       0x39 ./obj/printf.o
 .ARM.attributes
                0x0000035b       0x34 d:/ahl-gec-ide(4.20)/gcc/bin/../lib/gcc/arm-none-eabi/7.2.1/../../../../arm-none-eabi/lib/thumb/v7e-m/fpv4-sp/hard\libc_nano.a(lib_a-exit.o)
 .ARM.attributes
                0x0000038f       0x34 d:/ahl-gec-ide(4.20)/gcc/bin/../lib/gcc/arm-none-eabi/7.2.1/../../../../arm-none-eabi/lib/thumb/v7e-m/fpv4-sp/hard\libc_nano.a(lib_a-impure.o)
 .ARM.attributes
                0x000003c3       0x34 d:/ahl-gec-ide(4.20)/gcc/bin/../lib/gcc/arm-none-eabi/7.2.1/../../../../arm-none-eabi/lib/thumb/v7e-m/fpv4-sp/hard\libc_nano.a(lib_a-init.o)
 .ARM.attributes
                0x000003f7       0x34 d:/ahl-gec-ide(4.20)/gcc/bin/../lib/gcc/arm-none-eabi/7.2.1/../../../../arm-none-eabi/lib/thumb/v7e-m/fpv4-sp/hard\libc_nano.a(lib_a-memcpy-stub.o)
 .ARM.attributes
                0x0000042b       0x34 d:/ahl-gec-ide(4.20)/gcc/bin/../lib/gcc/arm-none-eabi/7.2.1/../../../../arm-none-eabi/lib/thumb/v7e-m/fpv4-sp/hard\libc_nano.a(lib_a-memset.o)
 .ARM.attributes
                0x0000045f       0x20 d:/ahl-gec-ide(4.20)/gcc/bin/../lib/gcc/arm-none-eabi/7.2.1/../../../../arm-none-eabi/lib/thumb/v7e-m/fpv4-sp/hard\libc_nano.a(lib_a-strcmp.o)
 .ARM.attributes
                0x0000047f       0x1b d:/ahl-gec-ide(4.20)/gcc/bin/../lib/gcc/arm-none-eabi/7.2.1/../../../../arm-none-eabi/lib/thumb/v7e-m/fpv4-sp/hard\libc_nano.a(lib_a-strlen.o)
 .ARM.attributes
                0x0000049a       0x34 d:/ahl-gec-ide(4.20)/gcc/bin/../lib/gcc/arm-none-eabi/7.2.1/../../../../arm-none-eabi/lib/thumb/v7e-m/fpv4-sp/hard\libc_nano.a(lib_a-strncmp.o)
 .ARM.attributes
                0x000004ce       0x22 d:/ahl-gec-ide(4.20)/gcc/bin/../lib/gcc/arm-none-eabi/7.2.1/thumb/v7e-m/fpv4-sp/hard\libgcc.a(_arm_addsubdf3.o)
 .ARM.attributes
                0x000004f0       0x22 d:/ahl-gec-ide(4.20)/gcc/bin/../lib/gcc/arm-none-eabi/7.2.1/thumb/v7e-m/fpv4-sp/hard\libgcc.a(_arm_muldivdf3.o)
 .ARM.attributes
                0x00000512       0x22 d:/ahl-gec-ide(4.20)/gcc/bin/../lib/gcc/arm-none-eabi/7.2.1/thumb/v7e-m/fpv4-sp/hard\libgcc.a(_arm_cmpdf2.o)
 .ARM.attributes
                0x00000534       0x22 d:/ahl-gec-ide(4.20)/gcc/bin/../lib/gcc/arm-none-eabi/7.2.1/thumb/v7e-m/fpv4-sp/hard\libgcc.a(_arm_fixunsdfsi.o)
 .ARM.attributes
                0x00000556       0x22 d:/ahl-gec-ide(4.20)/gcc/bin/../lib/gcc/arm-none-eabi/7.2.1/thumb/v7e-m/fpv4-sp/hard\libgcc.a(_aeabi_uldivmod.o)
 .ARM.attributes
                0x00000578       0x34 d:/ahl-gec-ide(4.20)/gcc/bin/../lib/gcc/arm-none-eabi/7.2.1/thumb/v7e-m/fpv4-sp/hard\libgcc.a(_fixunsdfdi.o)
 .ARM.attributes
                0x000005ac       0x34 d:/ahl-gec-ide(4.20)/gcc/bin/../lib/gcc/arm-none-eabi/7.2.1/thumb/v7e-m/fpv4-sp/hard\libgcc.a(_udivmoddi4.o)
 .ARM.attributes
                0x000005e0       0x22 d:/ahl-gec-ide(4.20)/gcc/bin/../lib/gcc/arm-none-eabi/7.2.1/thumb/v7e-m/fpv4-sp/hard\libgcc.a(_dvmd_tls.o)
 .ARM.attributes
                0x00000602       0x34 d:/ahl-gec-ide(4.20)/gcc/bin/../lib/gcc/arm-none-eabi/7.2.1/../../../../arm-none-eabi/lib/thumb/v7e-m/fpv4-sp/hard\libnosys.a(_exit.o)
 .ARM.attributes
                0x00000636       0x34 d:/ahl-gec-ide(4.20)/gcc/bin/../lib/gcc/arm-none-eabi/7.2.1/thumb/v7e-m/fpv4-sp/hard/crtend.o
 .ARM.attributes
                0x0000066a       0x22 d:/ahl-gec-ide(4.20)/gcc/bin/../lib/gcc/arm-none-eabi/7.2.1/thumb/v7e-m/fpv4-sp/hard/crtn.o

.comment        0x00000000       0x7e
 .comment       0x00000000       0x7e ./obj/emuart.o
                                 0x7f (size before relaxing)
 .comment       0x0000007e       0x7f ./obj/systick.o
 .comment       0x0000007e       0x7f ./obj/system_msp432p401r.o
 .comment       0x0000007e       0x7f ./obj/startup_msp432p401r_gcc.o
 .comment       0x0000007e       0x7f ./obj/main.o
 .comment       0x0000007e       0x7f ./obj/flash.o
 .comment       0x0000007e       0x7f ./obj/gpio.o
 .comment       0x0000007e       0x7f ./obj/wdog.o
 .comment       0x0000007e       0x7f ./obj/pwm.o
 .comment       0x0000007e       0x7f ./obj/gec.o
 .comment       0x0000007e       0x7f ./obj/uart.o
 .comment       0x0000007e       0x7f ./obj/isr.o
 .comment       0x0000007e       0x7f ./obj/printf.o

.debug_info     0x00000000     0x9e78
 .debug_info    0x00000000      0xc8f ./obj/emuart.o
 .debug_info    0x00000c8f      0x584 ./obj/systick.o
 .debug_info    0x00001213      0xd6a ./obj/system_msp432p401r.o
 .debug_info    0x00001f7d      0xa73 ./obj/startup_msp432p401r_gcc.o
 .debug_info    0x000029f0      0xa6b ./obj/main.o
 .debug_info    0x0000345b     0x1096 ./obj/flash.o
 .debug_info    0x000044f1     0x1547 ./obj/gpio.o
 .debug_info    0x00005a38      0x290 ./obj/wdog.o
 .debug_info    0x00005cc8      0x9e6 ./obj/pwm.o
 .debug_info    0x000066ae      0xc4a ./obj/gec.o
 .debug_info    0x000072f8     0x11f6 ./obj/uart.o
 .debug_info    0x000084ee      0xac8 ./obj/isr.o
 .debug_info    0x00008fb6      0xec2 ./obj/printf.o

.debug_abbrev   0x00000000     0x1b4d
 .debug_abbrev  0x00000000      0x29d ./obj/emuart.o
 .debug_abbrev  0x0000029d      0x150 ./obj/systick.o
 .debug_abbrev  0x000003ed      0x115 ./obj/system_msp432p401r.o
 .debug_abbrev  0x00000502      0x201 ./obj/startup_msp432p401r_gcc.o
 .debug_abbrev  0x00000703      0x203 ./obj/main.o
 .debug_abbrev  0x00000906      0x279 ./obj/flash.o
 .debug_abbrev  0x00000b7f      0x308 ./obj/gpio.o
 .debug_abbrev  0x00000e87       0xfd ./obj/wdog.o
 .debug_abbrev  0x00000f84      0x166 ./obj/pwm.o
 .debug_abbrev  0x000010ea      0x24b ./obj/gec.o
 .debug_abbrev  0x00001335      0x2fe ./obj/uart.o
 .debug_abbrev  0x00001633      0x266 ./obj/isr.o
 .debug_abbrev  0x00001899      0x2b4 ./obj/printf.o

.debug_aranges  0x00000000      0x1a0
 .debug_aranges
                0x00000000       0x20 ./obj/emuart.o
 .debug_aranges
                0x00000020       0x20 ./obj/systick.o
 .debug_aranges
                0x00000040       0x20 ./obj/system_msp432p401r.o
 .debug_aranges
                0x00000060       0x20 ./obj/startup_msp432p401r_gcc.o
 .debug_aranges
                0x00000080       0x20 ./obj/main.o
 .debug_aranges
                0x000000a0       0x20 ./obj/flash.o
 .debug_aranges
                0x000000c0       0x20 ./obj/gpio.o
 .debug_aranges
                0x000000e0       0x20 ./obj/wdog.o
 .debug_aranges
                0x00000100       0x20 ./obj/pwm.o
 .debug_aranges
                0x00000120       0x20 ./obj/gec.o
 .debug_aranges
                0x00000140       0x20 ./obj/uart.o
 .debug_aranges
                0x00000160       0x20 ./obj/isr.o
 .debug_aranges
                0x00000180       0x20 ./obj/printf.o

.debug_line     0x00000000     0x28ae
 .debug_line    0x00000000      0x31d ./obj/emuart.o
 .debug_line    0x0000031d      0x1f8 ./obj/systick.o
 .debug_line    0x00000515      0x272 ./obj/system_msp432p401r.o
 .debug_line    0x00000787      0x35a ./obj/startup_msp432p401r_gcc.o
 .debug_line    0x00000ae1      0x382 ./obj/main.o
 .debug_line    0x00000e63      0x3ad ./obj/flash.o
 .debug_line    0x00001210      0x392 ./obj/gpio.o
 .debug_line    0x000015a2      0x203 ./obj/wdog.o
 .debug_line    0x000017a5      0x24a ./obj/pwm.o
 .debug_line    0x000019ef      0x3ad ./obj/gec.o
 .debug_line    0x00001d9c      0x30f ./obj/uart.o
 .debug_line    0x000020ab      0x390 ./obj/isr.o
 .debug_line    0x0000243b      0x473 ./obj/printf.o

.debug_str      0x00000000     0x1a84
 .debug_str     0x00000000      0x66e ./obj/emuart.o
                                0x708 (size before relaxing)
 .debug_str     0x0000066e      0x38f ./obj/systick.o
                                0x58a (size before relaxing)
 .debug_str     0x000009fd      0x843 ./obj/system_msp432p401r.o
                                0xaed (size before relaxing)
 .debug_str     0x00001240       0xf0 ./obj/startup_msp432p401r_gcc.o
                                0x6e7 (size before relaxing)
 .debug_str     0x00001330       0x6e ./obj/main.o
                                0x6ac (size before relaxing)
 .debug_str     0x0000139e       0xe0 ./obj/flash.o
                                0xa12 (size before relaxing)
 .debug_str     0x0000147e      0x1c6 ./obj/gpio.o
                                0xb0a (size before relaxing)
 .debug_str     0x00001644       0x33 ./obj/wdog.o
                                0x2bb (size before relaxing)
 .debug_str     0x00001677      0x109 ./obj/pwm.o
                                0x45a (size before relaxing)
 .debug_str     0x00001780       0x42 ./obj/gec.o
                                0x6f5 (size before relaxing)
 .debug_str     0x000017c2       0xf2 ./obj/uart.o
                                0xa95 (size before relaxing)
 .debug_str     0x000018b4       0x77 ./obj/isr.o
                                0x6e7 (size before relaxing)
 .debug_str     0x0000192b      0x159 ./obj/printf.o
                                0x761 (size before relaxing)

.debug_frame    0x00000000      0xf3c
 .debug_frame   0x00000000      0x150 ./obj/emuart.o
 .debug_frame   0x00000150       0x60 ./obj/systick.o
 .debug_frame   0x000001b0       0x60 ./obj/system_msp432p401r.o
 .debug_frame   0x00000210       0x54 ./obj/startup_msp432p401r_gcc.o
 .debug_frame   0x00000264       0x30 ./obj/main.o
 .debug_frame   0x00000294      0x19c ./obj/flash.o
 .debug_frame   0x00000430      0x1c8 ./obj/gpio.o
 .debug_frame   0x000005f8       0x80 ./obj/wdog.o
 .debug_frame   0x00000678       0x90 ./obj/pwm.o
 .debug_frame   0x00000708       0x84 ./obj/gec.o
 .debug_frame   0x0000078c      0x21c ./obj/uart.o
 .debug_frame   0x000009a8       0xa4 ./obj/isr.o
 .debug_frame   0x00000a4c      0x17c ./obj/printf.o
 .debug_frame   0x00000bc8       0x28 d:/ahl-gec-ide(4.20)/gcc/bin/../lib/gcc/arm-none-eabi/7.2.1/../../../../arm-none-eabi/lib/thumb/v7e-m/fpv4-sp/hard\libc_nano.a(lib_a-exit.o)
 .debug_frame   0x00000bf0       0x2c d:/ahl-gec-ide(4.20)/gcc/bin/../lib/gcc/arm-none-eabi/7.2.1/../../../../arm-none-eabi/lib/thumb/v7e-m/fpv4-sp/hard\libc_nano.a(lib_a-init.o)
 .debug_frame   0x00000c1c       0x28 d:/ahl-gec-ide(4.20)/gcc/bin/../lib/gcc/arm-none-eabi/7.2.1/../../../../arm-none-eabi/lib/thumb/v7e-m/fpv4-sp/hard\libc_nano.a(lib_a-memcpy-stub.o)
 .debug_frame   0x00000c44       0x20 d:/ahl-gec-ide(4.20)/gcc/bin/../lib/gcc/arm-none-eabi/7.2.1/../../../../arm-none-eabi/lib/thumb/v7e-m/fpv4-sp/hard\libc_nano.a(lib_a-memset.o)
 .debug_frame   0x00000c64       0x20 d:/ahl-gec-ide(4.20)/gcc/bin/../lib/gcc/arm-none-eabi/7.2.1/../../../../arm-none-eabi/lib/thumb/v7e-m/fpv4-sp/hard\libc_nano.a(lib_a-strcmp.o)
 .debug_frame   0x00000c84       0x28 d:/ahl-gec-ide(4.20)/gcc/bin/../lib/gcc/arm-none-eabi/7.2.1/../../../../arm-none-eabi/lib/thumb/v7e-m/fpv4-sp/hard\libc_nano.a(lib_a-strncmp.o)
 .debug_frame   0x00000cac       0xac d:/ahl-gec-ide(4.20)/gcc/bin/../lib/gcc/arm-none-eabi/7.2.1/thumb/v7e-m/fpv4-sp/hard\libgcc.a(_arm_addsubdf3.o)
 .debug_frame   0x00000d58       0x50 d:/ahl-gec-ide(4.20)/gcc/bin/../lib/gcc/arm-none-eabi/7.2.1/thumb/v7e-m/fpv4-sp/hard\libgcc.a(_arm_muldivdf3.o)
 .debug_frame   0x00000da8       0xc4 d:/ahl-gec-ide(4.20)/gcc/bin/../lib/gcc/arm-none-eabi/7.2.1/thumb/v7e-m/fpv4-sp/hard\libgcc.a(_arm_cmpdf2.o)
 .debug_frame   0x00000e6c       0x24 d:/ahl-gec-ide(4.20)/gcc/bin/../lib/gcc/arm-none-eabi/7.2.1/thumb/v7e-m/fpv4-sp/hard\libgcc.a(_arm_fixunsdfsi.o)
 .debug_frame   0x00000e90       0x2c d:/ahl-gec-ide(4.20)/gcc/bin/../lib/gcc/arm-none-eabi/7.2.1/thumb/v7e-m/fpv4-sp/hard\libgcc.a(_aeabi_uldivmod.o)
 .debug_frame   0x00000ebc       0x2c d:/ahl-gec-ide(4.20)/gcc/bin/../lib/gcc/arm-none-eabi/7.2.1/thumb/v7e-m/fpv4-sp/hard\libgcc.a(_fixunsdfdi.o)
 .debug_frame   0x00000ee8       0x34 d:/ahl-gec-ide(4.20)/gcc/bin/../lib/gcc/arm-none-eabi/7.2.1/thumb/v7e-m/fpv4-sp/hard\libgcc.a(_udivmoddi4.o)
 .debug_frame   0x00000f1c       0x20 d:/ahl-gec-ide(4.20)/gcc/bin/../lib/gcc/arm-none-eabi/7.2.1/../../../../arm-none-eabi/lib/thumb/v7e-m/fpv4-sp/hard\libnosys.a(_exit.o)
